:100000000C9443170C946F170C946F170C946F1784
:100010000C946F170C946F170C946F170C946F1748
:100020000C946F170C946F170C946F170C946F1738
:100030000C946F170C947F2F0C946F170C946F1700
:100040000C946F170C946F170C946F170C946F1718
:100050000C946F170C946F170C946F170C946F1708
:100060000C946F170C946F170C946F170C946F17F8
:10007000000002060000FB00FF000000F405030C76
:1000800005040C05030C05040C05050000FF000029
:10009000FF000002090000F10400F900FF01000167
:1000A0000A0000E20201050101030101010205004D
:1000B00000FF000000E702030C04050000FF000041
:1000C00000F100085A0204030204040204050204B9
:1000D0000602050000FF010001010007900000E298
:1000E00008050000FF000002080107C80106000122
:1000F00000E700FF010001000007A00000EC010084
:10010000FE00010100FF010001030000E2030106FF
:1001100004010903050000FF000002010107C801F6
:1001200006000100EC00FF000002040000F10400E2
:10013000F900FF000002010000F100FF010000EDE6
:1001400000010602010100FF010000EC00010201B4
:1001500007000207FF00010300FF0000020800077C
:10016000640100140500F700FF000002090000F11F
:1001700000FF000002040000F800085003084E03CE
:10018000085402084C02085802084A01085C0000A2
:10019000FC03086003085A03086003085A03086058
:1001A00003085A01050000FF000002040000FB00E4
:1001B000083E0103020103020103020103020103DD
:1001C0000201040A01030201030201030201030206
:1001D00001030201040201030201030201030201FF
:1001E000030201030201040A0103020103020103E5
:1001F00002010302010302010405010302010302DB
:1002000001030201030201030201040501030201CB
:1002100003020103020103020103020104050103B9
:1002200002010302010302010302010302010500AE
:1002300000FF0000020300085602040A020408023C
:100240000406020404020402000842020305020438
:10025000020203050203050204020203050000F87E
:10026000040305040405040305040405040305044C
:10027000040504030501050000FF0000020400005E
:10028000FB00083401030201030401030601040A10
:1002900001030201030401030601040A0103020130
:1002A0000304010306010405010302010304010321
:1002B0000602030202030402030603040503030209
:1002C00003030403030604040504030204030404F3
:1002D000030601050000FF000007000402040007F8
:1002E000FF000990000A3C0000FB010850030305D1
:1002F00003040503030503040503030503040503C1
:1003000003050304050303050304050303050304B0
:100310000503030503050000FF00000700040204B5
:100320000007FF000990000A3C0000FB010853038E
:100330000305030405030305030405030305030480
:10034000050303050304050303050304050303056F
:1003500003040503030503050000FF000007000474
:1003600002040007FF000990000A3C0000FB01089E
:1003700056030305030405030305030405030305EE
:100380000304050303050304050303050304050330
:10039000030503040503030503050000FF00000730
:1003A000000402040007FF000990000A3C0000FB63
:1003B00001085903030503040503030503040503AA
:1003C00003050304050303050304050303050304F0
:1003D0000503030503040503030503050000FF00EF
:1003E0000002020106000100E000FF00000201011E
:1003F00006000100E000FF00000208010600010005
:10040000E000FF000002050106000100E000FF001F
:100410000002090106000100E000FF700079008E73
:100420000091009D00B200BE00D600E500F4000679
:10043000011801270133013C0148015A0169017289
:1004400001A80132027A02D70219035B039D03DF80
:1004500003EB03F70303040F040000000000000097
:10046000000000000000000000000000000000008C
:10047000000000000000000000000000000000007C
:100480000000000000000000000000380000000034
:1004900038383800000030303008000000200808EC
:1004A0000000002008000000000008000000001804
:1004B000000000000000080000383800383800381C
:1004C00038083838083008083008080008000008E4
:1004D000000000000000000000000000000000001C
:1004E000000000000000000000000000000000000C
:1004F000380038000030303030300000200820084C
:1005000008002008200800181818181800001808FB
:10051000180808000008000800000038000000006B
:100520003838383800300030080808002020200013
:1005300000000020002000181818180008000818F3
:1005400008080000000008000038380000000038EB
:1005500038080038000008083000080000200008B3
:10056000000020000800001800081818000008000B
:10057000181808000000000808003838000000388B
:100580000008380000300830000800002000080093
:10059000002000200020001808001800080018188B
:1005A00000180000000808000800383800000000AB
:1005B00000380800000030000800000000080000BB
:1005C000000000000000000000000000000000002B
:1005D00000000000000000000000000038000000E3
:1005E000003800080000300008000000200800006B
:1005F00000002008000000000018000000000000BB
:100600001800000000000008000038000000000092
:10061000003800000000000030000000000020084A
:10062000000000002008000000180008000018006A
:1006300008000000000800000000000000000000AA
:10064000003800000030003008300000202020007A
:1006500008200020082000000818080008000000FA
:100660000800000000000000000000000000000082
:10067000003800000000003008000020202020206A
:100680000000002008080800001808000000000012
:100690000800000000000000000000000000000052
:1006A000000000000000000000000000000000004A
:1006B00000002020000000000018080000001800C2
:1006C000080000000008000000000000000000001A
:1006D000000000000000000000000020202020207A
:1006E00000000808080808000000000000000000E2
:1006F00000000000000000000000000000000000FA
:1007000000000000000000000000000000000000E9
:100710000000000000000000181800000000181879
:1007200008000000000808000000000000000000B1
:100730000000003800000000300008000020000821
:100740000000200008000018000800000000080059
:1007500000000000000000000000777777000077BD
:1007600000010177002701002727011E011E001E3E
:10077000011E1E00011E010C0101000C01000C0CE9
:100780000C000100000101010000007700000000E2
:10079000777701000000002701000000001E010023
:1007A0000000001E01000000000C010000000C0C05
:1007B0000C0000000001010100007777770000774E
:1007C00000010177000001000027010000001E0069
:1007D0000100001E000100000C000100000C0C0CC8
:1007E0000C0C000001010101017777777777000099
:1007F00001017701010000270001000000001E0038
:1008000000000000001E000C0000000C01000C0C99
:100810000C00010000010101000000007700000051
:1008200000777701000027002701001E00011E014C
:10083000001E1E1E1E1E000001010C010100000012
:100840000C010000000000010077777777770077D0
:100850000101010101272727270000000101011ED6
:1008600000000000001E010C0000000C01000C0C38
:100870000C0001000001010100000077770000007A
:1008800077000101002700010000001E1E1E1E004F
:10089000001E0101011E000C0100000C01000C0CE7
:1008A0000C000100000101010077777777770000E5
:1008B000010101770100000027000100001E000176
:1008C00000001E00010000000C01000000000C01EF
:1008D000000000000001000000007777770000773B
:1008E0000001017700270100002701001E1E1E00E5
:1008F000011E0001011E000C0100000C01000C0C87
:100900000C000100000101010000777777000077FB
:100910000001017700270100002701001E1E1E1E96
:1009200001000001011E010000000C0001000C0C80
:1009300000010000000101000000000000000000B4
:1009400038380000000030300800000000080800BF
:100950000000202000000000181808000000000817
:10096000080000000000000000000000000000007F
:10097000383800000000303008000000000808008F
:1009800000002020000000000018080000001800EF
:10099000080000000008000000000000380000000F
:1009A000003800080000380008000020000800009F
:1009B00000002000000000000018000000000000FF
:1009C0001800000000000008000000000000000007
:1009D0000000000000303030303000000808080807
:1009E0000820202020200000080808080800000037
:1009F00000000000000000000000380000000000BF
:100A0000003800000000000030000000000000205E
:100A10000000000020000800001800080000180076
:100A200008000000000800000000383838000038D6
:100A3000000808380000080000300800000020000E
:100A40000800002000080000000008000000001856
:100A500000000000000008000000383838000038AE
:100A6000000808380000080000300800202000209E
:100A7000082000200820081808180818080018186E
:100A8000180008000008080800003838380000384E
:100A90000008083800300800003008200800002056
:100AA0000820202020200818080808180818080026
:100AB00000180800080000000838383838000038EE
:100AC00008080838003008000030082020202000E6
:100AD000082008080820001808000018081818182E
:100AE00018000800080808080000383838000038E6
:100AF0000008083800300800000008200800000046
:100B00000020080000000018080000180000181855
:100B100018000800000808080038383800000038BD
:100B200008083800003008000030002008000020CD
:100B300008200800002008180800180008181818D5
:100B40000008000008080800003838383838003835
:100B500008080808083008000000002020202000B5
:100B600000200808080800180800000000181818DD
:100B700018180000080808080838383838380038CD
:100B80000808080808300800000000202020200085
:100B900000200808080800180800000000180800D5
:100BA000000000000800000000003838380000385D
:100BB0000008083800300800000008200820202025
:100BC000002008000820081808000018080018185D
:100BD0001800080000080808003800000038003835
:100BE00008000038083008000030082020202020AD
:100BF000082008080820081808000018081808002D
:100C0000001808000800000008003838380000000C
:100C1000003808080000003008000000002008002C
:100C2000000000200800000000180800000018184C
:100C300018000000000808080000383838000000DC
:100C400000380808000000300800000000200800FC
:100C5000000000200800000000180800001818001C
:100C600008000000080800000038000000380038C4
:100C70000800380008300830000800202000080074
:100C800000200820000000180800180000180800C4
:100C900000180000080000000838000000000038BC
:100CA00008000000003008000000002008000000DC
:100CB00000200800000000180800000000181818A4
:100CC0001818000008080808083800000038003824
:100CD0003800383808300830003008200820082054
:100CE0000820080008200818080000180818080044
:100CF000001808000800000008380000003800381C
:100D0000080000380830300000300820082000209B
:100D100008200800202008180800001808180800FB
:100D200000180800080000000800383838000038B3
:100D300000080838003008000030082008000020B3
:100D400008200800002008180800001808001818DB
:100D50001800080000080808003838383800003843
:100D60000808083800300800003008202020200043
:100D700008200808080800180800000000180800EB
:100D8000000000000800000000003838380000387B
:100D90000008083800300800003008200800002053
:100DA000082008200020081808001800080018185B
:100DB00000180000000808000838383838000038EB
:100DC00008080838003008000030082020202000E3
:100DD000082008200808001808001800001808005B
:100DE00000180000080000000800383838380038C3
:100DF000000808080830080000000000202020003B
:100E0000000000080820000000000018081818184A
:100E1000180008000808080800383838383800007A
:100E20000838080808000038080000000020080002
:100E30000000002008000000001808000000001852
:100E400008000000000008000038000000380038EA
:100E50000800003808300800003008200800002092
:100E600008200800002008180800001808001818BA
:100E70001800080000080808003800000038003892
:100E80000800003808300800003008200800002062
:100E900008200800002008001800180008000018AA
:100EA000000800000000080000380000003800388A
:100EB0000800003808300800003008200800002032
:100EC0000820082000200818081808180800180032
:100ED000180008000008000800380000003800383A
:100EE000080000380800300030000800002000082A
:100EF000000020002000001800080018001808005A
:100F00000018080008000000083800000038003809
:100F100008000038083008000030080020002000D9
:100F20000800002000080000001808000000001859
:100F30000800000000000800003838383838000089
:100F400008080838080000003000080000200008E9
:100F50000000200008000018000800000018181801
:100F600018180000080808080800003838000000B9
:100F700038000800000030080000002000080000D1
:100F80000000200000000000180800000000001809
:100F900018000000000008080000003838000000B9
:100FA0003800003800380038380038380038000081
:100FB0003838003838003800380000380000003871
:100FC0003800000000000000000038380000000079
:100FD0000008380000000000300800000000002079
:100FE0000000000020000800000018080000181889
:100FF000000800000008080000C7C7C7C7C7C7C768
:10100000C7C7C7C7C7C7C7C7C7C7C7C7C7C7C7C770
:10101000C7C7C7C7C7C7C7C7C7C7C7C7C7C7C7C760
:10102000C7C7C7C7C7C7C7C7C700000000000000C1
:1010300000000000000000000000000000000000B0
:1010400000000000000000000000000000000000A0
:10105000000000000000000000000000000000038D
:101060000003030303030003030303030003030359
:101070000300000000000003030300030303030355
:10108000000303030303000303010C2121010303F5
:10109000313131210131317C7C31212131317C31BF
:1010A0003121213131312119212121212103191926
:1010B000211903010119190301010C0C0301030398
:1010C00001030103010C01010C0C03010C0C0303CF
:1010D0000C030103010C03010303030101030C01D1
:1010E000010C03010103030301010C373701030362
:1010F0003F3F3F37013F3F7F7F3F37373F3F7F3F96
:101100003F37373F3F3F371C3737373737031C1CD4
:10111000371C0301011C1C0301010C04040103031F
:10112000060606040106060F0F06040406060F064F
:10113000060404060606040304040404040303036B
:10114000040303010101030301010C4444010303EF
:10115000C7C7C74401C7C7DFDFC74444C7C7DFC726
:10116000C74444C7C7C74443444444444403434377
:10117000444303010143430301010CC8C8010303B5
:10118000D8D8D8C801D8D8F3F3D8C8C8D8D8F3D895
:10119000D8C8C8D8D8D8C848C8C8C8C8C8034848D4
:1011A000C84803010148480301010C5B5B010303CC
:1011B000ADADAD5B01ADADFFFFAD5B5BADADFFAD0B
:1011C000AD5B5BADADAD5B095B5B5B5B5B03090975
:1011D0005B0903010109090301000000000000038D
:1011E00000030303030300030303030300030303D8
:1011F00003000000000000030389898989038940F6
:1012000040404003894089898900000000000003B4
:1012100000030303030300030303030300030303A7
:1012200003000000000000898989898989404040C5
:1012300040404089898989898900000000000003B5
:101240000003030303030003030303030003030377
:10125000030000000000008989890003034040402A
:1012600089030389894089030300894089000003B9
:101270008940890303038940890303038940890363
:1012800003008940890000038940890303038940E2
:10129000890303038940890303003838383800384C
:1012A0000008080808300803030303032020200374
:1012B0000300000808200303030300180818181887
:1012C00018030803080808080300383838000038F5
:1012D0000008083803300803030308200803030349
:1012E0000320080000000018080300180303181862
:1012F00018030803030808080300383838000038CA
:1013000000080838033008030330082008030320CE
:1013100008200800002008180803001808031818FF
:101320001803080303080808033838383800003861
:101330000808083803300803033008202020200361
:1013400008200820080800180803180303180803D9
:101350000018030308030003083838383838003809
:10136000080808080830080303030320202020038E
:1013700003200808080800180803000303181818B9
:1013800018180303080808080800000000000003FC
:101390000003030303030003030303202020202092
:1013A00003000808080808030303000303030303FA
:1013B0000003030303030003033838383800003800
:1013C00008080838033008030330082020202003D1
:1013D0000820080808080018080300030318080379
:1013E0000003030308030003033800000000003873
:1013F0000803030303300803030303200803030364
:101400000320080000000018080300030318181840
:10141000181803030808080808003838380000388E
:1014200000080838033008030330082008030320AD
:101430000820202020200818080808180818080389
:1014400000180803080300030838000000380038BB
:10145000080303380830080303300803200320037F
:101460000800002000080003031808030303031802
:1014700008030303030308030300007700000003CD
:10148000777701030303002701030303001E010311
:101490000300001E01000003030C010303030C0CF6
:1014A0000C0303030301010103000000000000031B
:1014B000383803030303303008030303000808032C
:1014C000030020200000000318180803030303088A
:1014D000080303030303000303008940890000039A
:1014E00089408903030389408989890389404040F1
:1014F0004000894089898903894089030303894021
:1015000089030303894089030300000000000003EE
:101510000003030303898989898989404040404049
:10152000408989898989890303030003030303032D
:101530000003030303030003030089408900000341
:101540008940890303898940890303404040890316
:101550000389894089000003894089030303894086
:1015600089030303894089030300777777000077B5
:1015700000010177030301030327010300031E0396
:101580000100001E000100030C030103030C0C0CFE
:101590000C0C030301010101010000898989890301
:1015A00089404040400389408989890389408903F3
:1015B00003008940890000038940890303038940AF
:1015C00089030303894089030389898989898940BB
:1015D0004040404040898989898989031E1E0C0C3E
:1015E0001E0C030C031E0C030C0C0C03030C1E033B
:1015F000031E0C03030C0C0C0389898900000040B6
:101600004040890303898940890303038940890392
:10161000030089408900000389408903030389404E
:10162000890303038940890303008940890000037B
:10163000894089030303894089030303894089039F
:101640000300894089000003894089898903894012
:10165000404040030389898989031E1E0C030C0C3A
:10166000030C030C031E03031E1E0C031E1E0C0C96
:101670001E0C030C031E0C8989898989894040400E
:10168000404040898989898989008940890000030F
:10169000894089030303894089030303894089033F
:1016A0000300894089000089894089030340404044
:1016B000890303898989000303010CF1F100030305
:1016C000F9F9F9F101F9F9FCFCF9F1F1F9F9FCF991
:1016D000F9F1F1F9F9F9F1E1F1F1F1F1F103E1E1F8
:1016E000F1E1030101E1E10301010C0C0C01030331
:1016F0001E1E1E0C011E1E27271E0C0C1E1E271E42
:101700001E0C0C1E1E1E0C030C0C0C0C0C030303F5
:101710000C030301010103030100000000000000AD
:1017200000000000000000000000000000000000B9
:1017300000000000000000898989898989404040B3
:10174000404040898989898989898989898989402D
:101750004040404040898989898989000000000013
:101760000000000000000000000000000000000079
:10177000000000000000000000898989000000408E
:101780004040890000898940890000008940890023
:1017900000008940890000008940890000008940DC
:1017A0008900000089408900008989408900004043
:1017B0004040890000898989000000000000000085
:1017C0000000000000000000000000000000000019
:1017D0000000000000000000000000000000000009
:1017E00000000000000000000000000000000000F9
:1017F00000000000000000898989898989404040F3
:1018000040404089894089898989894089898940FE
:101810004040404040898989898989000000000052
:1018200000000000000000000000000000000000B8
:101830000000000000000000000000898989890084
:101840008940404040008940898989008940890059
:10185000000089408900000089408900000089401B
:1018600089000000894089000038000000380038F5
:101870000800003808300800003008200800002068
:1018800008200800002008001800180008000018B0
:101890000008000000000800000000000000000038
:1018A0000000000000000000000000000000000038
:1018B000000000000000000000898989890089403B
:1018C00040404000894089898900894089000000A2
:1018D0008940890000008940890000008940890012
:1018E000000089408900008989408900004040400B
:1018F000890000898940890000010C0C0301030361
:1019000001040404040C040F040F0401040F040F69
:101910000403040F040F04010404040404030C0072
:10192000010003010100030001010C0C030103038A
:101930003F361B03010C363F361B01011B3F1B3F8B
:101940003603363F3F3F3F01361B3F3636033F36B7
:1019500036361B010103030301010C272701030392
:1019600027CFCF270127CF2727CF27CF270C032724
:10197000CF27CF2727CF270127CFCF2701030C273A
:10198000270C03010103030301010C0C03010303F2
:1019900001030103015B01010C0C5B5BE0F1FBF156
:1019A0005B035BE0F15B03015BE0E05B01035BE099
:1019B000E05B0301015B5B0301FFFF00000000FF30
:1019C000F57F000000FFECF57F00007FECFFD97F82
:1019D000007FECD9D924007FECD92400007FEC24CF
:1019E0000000002424000000002600070000000181
:1019F00000010001000100010001000100010001DF
:101A000000010001000100010001000100010001CE
:101A100000010001000100010001000100010001BE
:101A200000010001000100010001000100010001AE
:101A3000000100010001000000010001000200029D
:101A40000002000200020003000400030003000380
:101A50000004000300050005000500050005000363
:101A6000000600030003000600030007000700074C
:101A7000000700070003000800080008000800082D
:101A80000001000100010001000200030003000347
:101A9000000300030004000400030003000400032B
:101AA0000005000300030003000500030006000317
:101AB0000006000300030007000300030003000307
:101AC00000030008000300030003000300010001FD
:101AD00000010001000200020002000200020003F7
:101AE00000040003000400030004000300050005D7
:101AF00000050005000500030006000600030003C2
:101B000000030007000700070007000300030008A8
:101B100000080008000800080001000100010001A1
:101B2000000300030003000300020003000400039D
:101B30000003000400040003000500030003000389
:101B40000005000300060003000600030003000771
:101B5000000300030003000300030003000300036D
:101B60000003000800010001000100010002000262
:101B7000000200020002000300040003000300034F
:101B80000004000300050003000300030005000338
:101B9000000600030003000600030007000700071B
:101BA00000070007000300080008000800080008FC
:101BB000000100010000000100010001000100011E
:101BC000000100010001000100010001000100010D
:101BD00000010001000100010001000100010001FD
:101BE00000010001000100010001000100010001ED
:101BF00000010001000100010001000100010000DE
:101C00000026001C0001000100010009000A000A72
:101C1000000A000A000A000A000A000A000A000A74
:101C2000000A000A000A000A000A000A000A000A64
:101C3000000A000A000A000A000A000A000A000A54
:101C4000000A000A000A000A000B0001000100015E
:101C5000000100010001000C000D000E000F00103B
:101C600000110012001300140015001600110010DE
:101C7000000100170018000100010001000100012F
:101C8000000100010001000100010001000100014C
:101C900000010001000C0001000100010001000131
:101CA00000010019001A001A001A001A001A001A7E
:101CB000001A001A001A001A001A001A001A001A54
:101CC000001A001A001A001A001A001A001A001A44
:101CD000001A001A001A001A001A001A001A001A34
:101CE000001B000100010001000100010001000CC7
:101CF000000D000E000F0010001100120013001460
:101D000000150016001100100001001C0018000151
:101D100000010001000100010001000100010001BB
:101D2000000100010001000100010001000C0001A0
:101D300000010001001D001E001E001E001E001EEE
:101D4000001E001E001E001E001E001E001E001EA3
:101D5000001E001E001E001E001E001E001E001E93
:101D6000001E001E001E001E001E001E001E001E83
:101D7000001E001E001E001E001E001E001E001F72
:101D8000000C000300030003000300030003000332
:101D9000000300030003000300030003000300032B
:101DA000000300030003000300030003000300031B
:101DB000000300030003000300030003000300030B
:101DC00000030003000300030003000C000C0003E9
:101DD00000030003000300030003000300030003EB
:101DE00000030003000300030003000300030003DB
:101DF00000030003000300030003000300030003CB
:101E000000030003000300030003000300030003BA
:101E1000000300030003000C000C00030003000398
:101E2000000300030003000300030003000300039A
:101E3000000300030003000300030003000300038A
:101E4000000300030003000300030003000300037A
:101E5000000300030003000300030003000300036A
:101E60000003000C000C0003000300030003000348
:101E7000000300030003000300030003000300034A
:101E8000000300030003000300030003000300033A
:101E9000000300030003000300030003000300032A
:101EA0000003000300030003000300030003000C11
:101EB000000C000300030003000300030003000301
:101EC00000030003000300030003000300030003FA
:101ED00000030003000300030003000300030003EA
:101EE00000030003000300030003000300030003DA
:101EF00000030003000300030003000C000C0003B8
:101F000000030003000300030003000300030003B9
:101F100000030003000300030003000300030003A9
:101F20000003000300030003000300030003000399
:101F30000003000300030003000300030003000389
:101F4000000300030003000C000C00030003000367
:101F50000003000300030003000300030003000369
:101F60000003000300030003000300030003000359
:101F70000003000300030003000300030003000349
:101F80000003000300030003000300030003000339
:101F90000003000C000C0003000300030003000317
:101FA0000003000300030003000300030003000319
:101FB0000003000300030003000300030003000309
:101FC00000030003000300030003000300030003F9
:101FD0000003000300030003000300030003000CE0
:101FE000000C0003000300030003000300030003D0
:101FF00000030003000300030003000300030003C9
:1020000000030003000300030003000300030003B8
:1020100000030003000300030003000300030003A8
:1020200000030003000300030003000C000C000386
:102030000003000300030003000300030003000388
:102040000003000300030003000300030003000378
:102050000003000300030003000300030003000368
:102060000003000300030003000300030003000358
:10207000000300030003000C000C00030003000336
:102080000003000300030003000300030003000338
:102090000003000300030003000300030003000328
:1020A0000003000300030003000300030003000318
:1020B0000003000300030003000300030003000308
:1020C0000003000C000C00030003000300030003E6
:1020D00000030003000300030003000300030003E8
:1020E00000030003000300030003000300030003D8
:1020F00000030003000300030003000300030003C8
:102100000003000300030003000300030003000CAE
:10211000000C00030003000300030003000300039E
:102120000003000300030003000300030003000397
:102130000003000300030003000300030003000387
:102140000003000300030003000300030003000377
:1021500000030003000300030003000C000C000355
:102160000003000300030003000300030003000357
:102170000003000300030003000300030003000347
:102180000003000300030003000300030003000337
:102190000003000300030003000300030003000327
:1021A000000300030003000C000C00030003000305
:1021B0000003000300030003000300030003000307
:1021C00000030003000300030003000300030003F7
:1021D00000030003000300030003000300030003E7
:1021E00000030003000300030003000300030003D7
:1021F0000003000C000C00030003000300030003B5
:1022000000030003000300030003000300030003B6
:1022100000030003000300030003000300030003A6
:102220000003000300030003000300030003000396
:102230000003000300030003000300030003000C7D
:10224000000C00030003000300030003000300036D
:102250000003000300030003000300030003000366
:102260000003000300030003000300030003000356
:102270000003000300030003000300030003000346
:1022800000030003000300030003000C000C000324
:102290000003000300030003000300030003000326
:1022A0000003000300030003000300030003000316
:1022B0000003000300030003000300030003000306
:1022C00000030003000300030003000300030003F6
:1022D000000300030003000C000C000300030003D4
:1022E00000030003000300030003000300030003D6
:1022F00000030003000300030003000300030003C6
:1023000000030003000300030003000300030003B5
:1023100000030003000300030003000300030003A5
:102320000003000C000C0003000300030003000383
:102330000003000300030003000300030003000385
:102340000003000300030003000300030003000375
:102350000003000300030003000300030003000365
:102360000003000300030003000300030003000C4C
:102370000020002100210021002100210021002156
:102380000021002100210021002100210021002145
:102390000021002100210021002100210021002135
:1023A0000021002100210021002100210021002125
:1023B0000021002100210021002100220001000154
:1023C0000001000100010001000100010001000105
:1023D00000010001000100010001000100010001F5
:1023E00000010001000100010001000100010001E5
:1023F00000010001000100010001000100010001D5
:1024000000010001000100010001000100010001C4
:1024100000010001000100010001000100010001B4
:1024200000010001000100010001000100010001A4
:102430000001000100010001000100010001000194
:102440000001000100010001000100010001000184
:1024500000010001003120504C415945520032200A
:10246000504C415945520047414D45204F50544929
:102470004F4E5300425241444C455920424F434332
:10248000555A5A49202D203230303800534E414B96
:102490004520434F4C4F52002D504C41594552203E
:1024A000313A002D504C4159455220323A00535494
:1024B000415254494E472053504545443A005354E5
:1024C000415254494E47204C454E4754483A0052D9
:1024D000455455524E0047414D45204F56455221D7
:1024E00000504C4159455220312057494E5321004C
:1024F000504C4159455220322057494E53210052E9
:10250000454400424C5545004C4947485420424CF4
:10251000554500475245454E004F52414E474500F4
:1025200053494C5645520059454C4C4F5700505555
:1025300052504C450052414E444F4D495A450000BF
:10254000000000000000000000000000000000008B
:10255000000000000000000000000000000000007B
:10256000000000000000000000000000000000006B
:10257000000000000000000000000000000000005B
:10258000000000000000000000000000000000004B
:10259000000049000000495252000052525C2D00D8
:1025A000000000000000000000000000000000002B
:1025B00040000000494A52004952525B1C52531CD1
:1025C00025241B2425251B0A0A2D1C12120A0A0089
:1025D00000000000000000404949494949525B5B46
:1025E0005B525B1C1C1312241C12090909120909F5
:1025F00009090A0A0A0A0A0A13120A0A12130A0025
:10260000000000000092525252525213121309005D
:102610001C0A1212401B65090A0009241B12000043
:10262000251C1C010025241C1C0024252424240016
:1026300000000000005249494000001B1352494964
:1026400000641C1C5B4A481C651C2552491C1C6507
:102650002464491C1C652564491C1C6D2E5C4900C2
:1026600000000000000000000000490000000053CE
:102670005200000053522500004A52252500005BFD
:10268000251300005B53000A1C095B1C657F374063
:1026900052522E2E1C525C2E251B1324251C1C125C
:1026A000002525120000121B0000132E37001B37D7
:1026B000372E2E37372E2E2E2E2E2E6E6E6E1C138C
:1026C00013120009131200001213130012251C1319
:1026D000132E371C131313361C131B1B1B25131C23
:1026E0001C1B1B1B1C1C1C1C1C1C1C1C1C1C13133F
:1026F00012121313001313131C000913131C0100EF
:1027000037131C13002E2E1C1C001C772E250013C3
:102710007F251C010A37241C1C0A2E2525090013BD
:102720002E242525252E252525252525252D2E2537
:102730001B2E2E251C1325251C1C1C1C011C1C13C8
:1027400000011C0A000165775C016E7F6E521B253B
:10275000256D1C524925251C1353001C1C1C524A74
:10276000001B135B5B000009525C0000005B5C0017
:102770000000001B0000000000000000000000132B
:102780005B7F776E6E136577766E6E1B65777676F8
:10279000761B5BBF76B67609136DBFB7B6001B120A
:1027A0005C76BF0000121B125B00000000090A6E7D
:1027B0006E6E77241C6E6E77251C1C6E776E1C1C4B
:1027C0001C76761C1C2425B765646D6D1B766D6DBB
:1027D0005B09125B5C5B125B641213131B12121C0D
:1027E0001C1C1C1C241C1C242525242425251B0002
:1027F000002513000064BF00096EBFBF6D6EBF6D82
:102800005B12135B12131209000901000000002E75
:102810001C0900096E010009767F7F12777F7F64B3
:1028200012BF775B121B095B121B0900001B09001A
:102830000000000000000000000000000000007F19
:102840007F5313130064121B0100001B12000000D1
:102850000000000000000000000000000000000078
:102860000000000000000000000000000000000068
:1028700000000000002600000026002F0000002FAE
:1028800000370000003700FF000000FF00BF00001D
:1028900000BF0037000037000000262600000000BF
:1028A0000000000000262626262600000000002F3B
:1028B000000000003700000000FF00000000BF0023
:1028C0000000003700000000002626262626000013
:1028D00000000000002626262626002F000000000B
:1028E00000370000000000FFFFFFFF0000BF0000F6
:1028F00000000037000000000026262626260000E3
:1029000000000000002626262600002F0000002FD1
:1029100000370000003700FFFFFFFF0000BF00008E
:1029200000BF0037000000370026262626000000E2
:102930000000000000000026262600002F00002FC7
:1029400000370000003700FF000000FF00BF00005C
:1029500000BF0037000037000026262600000000D8
:1029600000000000002600000026002F0000002FBD
:10297000000037003700000000FF00000000BF002B
:10298000BF000037000000370026000000260000CE
:102990000000000000000000000000000000000037
:1029A0000000000000000000000000000000000027
:1029B00000009B000000529BA400005B9B6D770011
:1029C0000000000000000000000000000000000007
:1029D0005B000000E4F6FF099BEDF6FFBFA4ADBF6E
:1029E000BFBFBF767F7FB7B7BF7F766EB7B7BF0079
:1029F000000000000000005BB6F6F6F6FFFFFFFFE8
:102A0000BFFFFFFFBFBFAEFFFFFFB7AD65FFFFB763
:102A1000B6AD65FFFFBFB7AE6EFFFFBFB7B76500CE
:102A20000000000000F6F6EDEDADA4B66D6D5C5251
:102A30006E6565655265765C5C52536E24655252D4
:102A40006E25255B52772D2525526E6E2D2525008E
:102A50000000000000A49B9B4900006564A49B92B9
:102A6000006D2525649349656E652E9B5224256D66
:102A700025655225246D2D655225256E2E64520044
:102A8000000000000000000000004A000000005BA1
:102A90009B0000005B5B2D0000525B2E2E00015B53
:102AA0002D1C01005C5B014A654A5B1C6E7F774907
:102AB0005B9B77776D5B65776E65656D2D25255C16
:102AC000522E25130949641C09095C7F7F091C7F6C
:102AD0007F777F777F77777F7F7776777F7F6E656A
:102AE0006E6EA4B6FF655BA4B7BFFF526DBFBFBFDC
:102AF000FF7FBFBFBFBFFFBFBFB7BFFFFF7FB7BF76
:102B0000BFFFFF6EB7BFBFFFFF77BFBFBFFFFFFFB6
:102B1000FFBFBFB75BFFFFBFBFA464FFFFBFADA494
:102B20007FFFFFBFA4BF7FFFBFADBFBFBFFFB6BF6B
:102B3000BFBF77F7BFBFBF7777FFBFBFBF64526D1F
:102B40007F6E2E2D2D7F766E6E6E2E777777762E9A
:102B50001C7F776E251C25776525251C096E6E1C4C
:102B60000949255B494A6E7F645377BF775B5C25D3
:102B70006E6E255B4A25651C1B5B002524245B5378
:102B8000001C1B5B5C00000A5B64000000646400C6
:102B90000000005C00000000000000000000005B7E
:102BA0005C7FBF77765C6D7FB777775C6D7FBF7733
:102BB000775C64BFBFBFBF0A5C6EBFBFBF00656408
:102BC0006DBFBF00005B6D646D00000000125B779D
:102BD00077777F6E6E77777F766D7677BF776D6E5E
:102BE00076BF7F6D6E767FBF7676BFBF76BFBFBF85
:102BF000B664ADADB6B6ADBFFF646DADB6AD6477CE
:102C0000BFBFBFFFFF77BFBFBFFFFF7FBFBFBFFF1C
:102C1000F6BFB7ADF6FFFFA4ADFFFFFFFFFFFFFF5D
:102C2000FFFFFFFFFFFFF6A4005B5200000000BFA4
:102C3000BFAD5B64BFB6ADADBFFFBFFFFFFFFFBF62
:102C400064FFFFBFB6765BFFBFBF5B0000FF5C00A9
:102C5000000000000000000000000000000000BFB5
:102C6000BF645C5C006E5C654900006D5B00000049
:102C70000000000000000000000000000000000054
:102C8000000000000000000000000000000000063E
:102C9000000400000001000200030004000500061B
:102CA000000700080009000A000B000C000D000ED0
:102CB000000F001000000011001200130014001596
:102CC0000016000600030000001700180019001A83
:102CD000001B001C001D001E001F00200021002200
:102CE0000023002400250026000000000002080048
:102CF000085504085A0000F8000990000A1E320521
:102D00000000FFEB2C0000000100020003000400A3
:102D10000501000101010201030104010502000295
:102D2000010202020302040205030003010302037D
:102D3000030304030504000401040204030404045F
:102D40000505000501050205030504050506000645
:102D5000010602060306040605070007010702072D
:102D6000030704070508000801080208030804080F
:102D7000050900090109020903090409050A000AF5
:102D8000010A020A030A040A050B000B010B020BDD
:102D9000030B040B050C000C010C020C030C040CBF
:102DA000050D000D010D020D030D040D050E000EA5
:102DB000010E020E030E040E050F000F010F020F8D
:102DC000030F040F0510001001100210031004106F
:102DD0000511001101110211031104110512001255
:102DE000011202120312041205130013011302133D
:102DF000031304130514001401140214031404141F
:102E00000515001501150215031504150516001604
:102E100001160216031604160517001701170217EC
:102E200003170417051800180118021803180418CE
:102E3000051900190119021903190419051A001AB4
:102E4000011A021A031A041A051B001B011B021B9C
:102E5000031B041B051C001C011C021C031C041C7E
:102E6000051D001D011D021D031D041D051E001E64
:102E7000011E021E031E041E051F001F011F021F4C
:102E8000031F041F050011241FBECFEFD0E1DEBFDA
:102E9000CDBF14BE88E10FB6F89480936000109205
:102EA00060000FBE11E0A0E0B1E0E4E3F4E602C090
:102EB00005900D92AC32B107D9F71EE0ACE2B1E05B
:102EC00001C01D92A431B107E1F70E9428260E949B
:102ED00082300E944C200E948D1F0C9418320C945A
:102EE00000008430910509F18530910548F4823065
:102EF0009105A9F083309105A8F4019769F409C000
:102F000086309105C1F08630910590F0079721F445
:102F100015C082E090E014C080E090E011C083E032
:102F200090E00EC084E090E00BC085E090E008C027
:102F300086E090E005C081E290E002C082E290E08D
:102F4000672B29F490932E0180932D01089590937F
:102F5000070180930601089580E00E94112090FDF2
:102F6000FBCF80E00E94112090FFFBCF80E00E9409
:102F7000112090FDFBCF08950E94423164E270E081
:102F80000E945E31039690930D0180930C010E9484
:102F9000423164E170E00E945E31059690930F012A
:102FA00080930E010895EF92FF920F931F93CF939A
:102FB000DF937B016115710529F41092B102C4E120
:102FC000D0E004C01092B202C6E1D0E08430910596
:102FD00009F46DC08530910568F48130910541F1A7
:102FE00081309105B8F082309105B9F1039709F06D
:102FF000CEC048C08630910509F483C08630910563
:1030000008F46AC08730910509F490C0089709F068
:10301000BEC0A1C000E210E021E030E04AE050E094
:10302000BE018EE190E00E94B32C43E155E2AAC0BC
:1030300000E210E021E030E04AE050E0BE018EE125
:1030400090E00E94B32C47E255E2BE018EE190E091
:103050000E94EE2C82E090E09CC000E210E021E0B3
:1030600030E04AE050E0BE018EE190E00E94B32CD7
:103070004FEF54E2BE018EE190E00E94EE2C83E01F
:1030800090E087C000E210E021E030E04AE050E04C
:10309000BE018EE190E00E94B32C4EE255E2BE01EB
:1030A0008EE190E00E94EE2C84E090E072C000E29D
:1030B00010E021E030E04AE050E0BE018EE190E017
:1030C0000E94B32C43E055E2BE018EE190E00E94E5
:1030D000EE2C85E090E05DC000E210E021E030E001
:1030E0004AE050E0BE018EE190E00E94B32C40E245
:1030F00055E2BE018EE190E00E94EE2C86E090E069
:1031000048C000E210E021E030E04AE050E0BE01BB
:103110008EE190E00E94B32C48E055E2BE018EE1C2
:1031200090E00E94EE2C81E290E033C000E210E0DB
:1031300021E030E04AE050E0BE018EE190E00E94E4
:10314000B32C49E155E2BE018EE190E00E94EE2CE5
:1031500082E290E01EC0E114F10421F481E080934A
:10316000B10203C081E08093B20200E210E021E0EE
:1031700030E04AE050E0BE018EE190E00E94B32CC6
:1031800045E355E2BE018EE190E00E94EE2C80E026
:1031900090E0EF2829F490932E0180932D0104C034
:1031A0009093070180930601DF91CF911F910F91BA
:1031B000FF90EF9008956F927F928F929F92AF92BF
:1031C000BF92CF92DF92EF92FF920F931F93CF9314
:1031D000DF93EC016A017B015901902E812E3C01A5
:1031E0000894610871089A01AB01602F712FC30127
:1031F0008A0D9B1D0E94842DD701C6010A97A10943
:10320000B1098A359105A105B10510F4229724C0B2
:10321000D701C60184569040A040B04084589340E6
:10322000A040B04010F4239717C0D701C601885EB4
:103230009340A040B04088529342A040B04010F468
:1032400024970AC080E1C81687E2D80680E0E80625
:1032500080E0F80638F0259700E310E021E030E048
:10326000AE0105C000E310E021E030E0A301692DCC
:10327000782DC5010E94B32CDF91CF911F910F9142
:10328000FF90EF90DF90CF90BF90AF909F908F9086
:103290007F906F9008950F931F9360910A01709132
:1032A0000B012091310130913201892B11F5629F80
:1032B000A001639F500D729F500D11244B5F5F4F13
:1032C00060E070E08091330190913401A09135016C
:1032D000B0913601480F591F6A1F7B1F409333017D
:1032E00050933401609335017093360101E010E092
:1032F00021C0629FA001639F500D729F500D112449
:103300004B5F5F4F60E070E0809137019091380132
:10331000A0913901B0913A01480F591F6A1F7B1FD4
:1033200040933701509338016093390170933A010B
:1033300003E010E026E130E087E090E00E94DB1837
:103340001F910F910895FF920F931F93CF93DF93D7
:1033500089319105B9F18A31910548F48830910598
:10336000F9F08231910529F1892B89F037C0823338
:103370009105F9F08333910518F44E9779F507C05C
:103380008334910569F08535910541F51BC080E3D3
:1033900090E0909311018093100185E090E01AC0B5
:1033A0008FE290E090931101809310018AE090E009
:1033B00011C081E390E090931101809310018BE0A4
:1033C00090E008C082E390E0909311018093100197
:1033D00084E190E09093320180933101C0910C011F
:1033E000D0910D0160910E0170910F010091AD021D
:1033F0001091AE02F0902C01A5E9B1E0E1EFF1E00F
:103400004DE250E02D913C9111972D5F3F4FC21737
:10341000D30749F48081918105966817790719F4DB
:103420004017510778F081E0F81679F4C217D307F6
:1034300061F48081918105966817790731F440170E
:10344000510718F40E94BC17C9CF41505040129741
:10345000329741155105B1F6C093040160930501FF
:1034600040911001509111018C2F0E946830DF9122
:10347000CF911F910F91FF9008950E94003045E574
:1034800054E26EE070E080E190E00E94EE2C4EE5A8
:1034900054E260E170E080E190E00E94EE2C47E6AB
:1034A00054E262E170E080E190E00E94EE2C44E79B
:1034B00054E268E170E08BE090E00E94EE2C49EE6F
:1034C00059E162E082E00E94FA2D08951F93182FBF
:1034D00046ED54E26FE070E08FE090E00E94EE2C49
:1034E00080912C01813069F4112319F440EF54E2EA
:1034F00002C041EE54E260E170E08DE090E00E9495
:10350000EE2C84E690E00E94472E0E943D1A1F9107
:1035100008952F923F924F925F926F927F928F9277
:103520009F92AF92BF92CF92DF92EF92FF920F9352
:103530001F93DF93CF93CDB7DEB763970FB6F894A1
:10354000DEBF0FBECDBF8091AB029091AC020E9456
:1035500047310E94BC170E94003080E090E022E2D8
:1035600030E0FC01E55CFE4F11821082FC01E9565F
:10357000FE4F31832083FC01ED50FE4F31832083C9
:10358000FC01E15BFD4F3183208302968A35910572
:1035900041F71092330110923401109235011092CC
:1035A00036011092370110923801109239011092B1
:1035B0003A018AE0809305018093040141E05CE1D7
:1035C00060E082E00E94FA2D01E010E026E130E0A8
:1035D00040E050E060E070E087E090E00E94DB189F
:1035E00003E010E026E130E040E050E060E070E011
:1035F00087E090E00E94DB1880E090E00E94A31931
:10360000198618861F821E822224332463E2462EE6
:10361000512C6624772488249924CC24DD24AA24E0
:10362000BB24EE24FF241D821C821D861C861B8663
:103630001A868091B102882351F00E94423168E0DD
:1036400070E00E945E3160E070E00E94711780912E
:10365000B202882351F00E94423168E070E00E947B
:103660005E3160E070E00E9471172E813F813093DF
:103670003E0120933D0130929A012092990150928F
:10368000F6014092F50170925202609251028091CF
:103690000201909103012C853D85280F391F30933D
:1036A000AE022093AD024A855B85840F951F9093EF
:1036B000B0028093AF0280E00E9411208C018091C3
:1036C0002C01813021F40E9411209987888707FFFF
:1036D00008C051E08516910421F088248A94982C22
:1036E0000AC006FF0BC08FEF88168FEF980631F0E7
:1036F00051E0852E912CCC24DD241DC005FF0AC08D
:1037000091E0C916D10431F088249924CC24CA94BC
:10371000DC2C11C004FF0BC0EFEFCE16EFEFDE067E
:1037200031F08824992441E0C42ED12C04C010FF2C
:1037300002C00E94AC1780912C018130D1F5F88530
:10374000F7FF08C021E0A216B10421F0AA24AA9430
:10375000BA2C0BC0388536FF0BC04FEFA4164FEFC5
:10376000B40631F031E0A32EB12CEE24FF2421C0A9
:10377000588555FF0AC081E0E816F10431F0AA240B
:10378000BB24EE24EA94FE2C14C0988594FF0BC051
:10379000EFEFEE16EFEFFE0631F0AA24BB2421E096
:1037A000E22EF12C06C02885398530FF02C00E9428
:1037B000AC174E815F814432510508F0D7C04C0DE3
:1037C0005D1D5F834E8354E12516310408F0CEC0A1
:1037D000280C391C84E24816510408F023C14E0C11
:1037E0005F1C94E16916710408F01CC16A0C7B1C13
:1037F000E091AD02F091AE02EE0FFF1FDF01A9567E
:10380000BE4F6C916B5FE55CFE4F808143E050E002
:103810008D5F0E94683080912C01813099F4E09195
:10382000AF02F091B002EE0FFF1FDF01A15BBD4FB1
:103830006C916B5FED50FE4F808143E050E08D5FF7
:103840000E9468300E94BC17E091AD02F091AE0278
:10385000FB83EA83F0912C01F9830091AF02109170
:10386000B00263E971E0AFEEB1E02BE432E03B8BF4
:103870002A8B47EA52E0598B488B2DE230E0FB015E
:10388000428153818E819F8184179507B9F4EA8123
:10389000FB812E173F0790F4F1E0CF16D10461F1C0
:1038A0008FEFC8168FEFD80639F19FEF89169FEF7B
:1038B000990611F1E1E08E169104F1F0E889F98999
:1038C0000280F381E02DFF87EE872E163F0609F078
:1038D0004FC0EA89FB8982819381EE81FF81E817DD
:1038E000F90709F045C08A819B812817390708F03C
:1038F0003FC099819130E1F512968D919C9113977B
:1039000028163906B9F4EA81FB812E173F0790F497
:10391000F1E0CF16D10451F14FEFC4164FEFD406AA
:1039200029F15FEF85165FEF950601F181E08816BA
:103930009104E1F0E889F98982819381281639069A
:1039400009F08CC0EA89FB89828193814E815F8175
:103950004817590709F082C08A819B8128173907C7
:1039600008F07CC09981913009F078C080E05BC09C
:10397000EA89FB898281938148165906A9F42017A8
:10398000310790F4F1E0EF16F10411F18FEFE81632
:103990008FEFF806E9F09FEFA9169FEFB906C1F087
:1039A000E1E0AE16B104A1F012968D919C911397AF
:1039B0006816790609F052C04416550609F04EC043
:1039C0002017310708F04AC0F981F13009F046C0EC
:1039D0008E859F8568167906A9F42017310790F423
:1039E00091E0E916F104F1F0EFEFEE16EFEFFE06CD
:1039F000C9F0FFEFAF16FFEFBF06A1F081E0A816F8
:103A0000B10481F012968D919C91139768167906F6
:103A100029F54416550611F520173107F8F4998158
:103A20009130E1F481E00E94661A63960FB6F89433
:103A3000DEBF0FBECDBFCF91DF911F910F91FF90E1
:103A4000EF90DF90CF90BF90AF909F908F907F903E
:103A50006F905F904F903F902F900895215030408D
:103A6000FB0180819181938382838D919C91119739
:103A700013969C938E931297EA89FB89808191819A
:103A800093838283E889F9898081918193838283FA
:103A90006250704012974A895B89425050405B8B5C
:103AA0004A8B3297F98BE88B2115310509F0E7CE67
:103AB00040912D0150912E014E5F5F4F622D6B5F43
:103AC0008E818D5F0E94683080912C01813061F47D
:103AD00040910601509107014E5F5F4F662D6B5F6D
:103AE000842D8D5F0E9468308091000190910101CA
:103AF000EBE0F0E0E81BF90BCF010E94472E80912C
:103B00000401482F50E08E819F810396841795070A
:103B100009F591012B5F3F4F8091050190E0281737
:103B20003907C1F48091AD029091AE028D9730F4C7
:103B30002C853D852F5F3F4F3D872C874C815D81D4
:103B40004F5F5F4F5D834C83CA010E94A31980E0E1
:103B500090E02AC0C20103968417950709F069CD49
:103B600093012B5F3F4F8091050190E028173907A3
:103B700009F05FCD80912C01813009F05ACD809100
:103B8000AF029091B0028D9728F48A859B850196AB
:103B90009B878A87EC81FD813196FD83EC83CF0181
:103BA0000E94A31981E090E00E944B1942CDDF9260
:103BB000EF92FF920F931F93CF93DF930E940030F9
:103BC00047E654E267E070E08EE090E00E94EE2C61
:103BD0004EEA54E26EE070E08FE090E00E94EE2C3E
:103BE0004EEB54E260E170E08FE090E00E94EE2C3A
:103BF0004CE854E262E170E08FE090E00E94EE2C2D
:103C000048E954E264E170E082E190E00E94EE2C29
:103C100043EA54E266E170E082E190E00E94EE2C1B
:103C20004FEC54E26CE070E08FE090E00E94EE2CEC
:103C300043E350E06CE08EE00E9468304091000168
:103C40006EE081E20E940A2D4091020160E181E272
:103C50000E940A2D60E070E080912F019091300168
:103C60000E94D31761E070E08091080190910901F2
:103C70000E94D31700E0DD2410E08091AB02909108
:103C8000AC0201969093AC028093AB0280E00E945C
:103C90001120EC0188709170892B11F180E00E9455
:103CA0001120892BD9F7112351F40E943D1ADF917D
:103CB000CF911F910F91FF90EF90DF9008951630F4
:103CC00079F440E050E062E18EE00E946830602FBD
:103CD0006C5E43E350E081E10E946830DD24D394C0
:103CE000D3FF17C080E00E941120892BD9F781E013
:103CF000D81679F4612F645F43E350E08EE00E94B0
:103D00006830602F6C5E40E050E081E10E946830D6
:103D1000DD24C4FF51C0123079F44091000150916C
:103D2000010147305105E0F44F5F5F4F50930101AF
:103D3000409300016EE010C0143091F440910201F4
:103D4000509103014930510558F44F5F5F4F509334
:103D500003014093020160E181E20E940A2D27C025
:103D6000002389F4163019F580912F0190913001CC
:103D700088309105E0F401969093300180932F01F3
:103D800060E070E012C0023091F4163081F480914E
:103D90000801909109018830910548F401969093AB
:103DA00009018093080161E070E00E94D31780E070
:103DB0000E941120892BD9F7C5FF57C01230B9F4E2
:103DC00040910001509101014230510520F14150D4
:103DD000504050930101409300016EE081E20E9447
:103DE0000A2D80E00E941120892BD9F739C01430A8
:103DF00091F440910201509103014530510558F072
:103E000041505040509303014093020160E181E230
:103E10000E940A2D25C0002381F4163009F58091F7
:103E20002F01909130010097D9F0019790933001C4
:103E300080932F0160E070E011C0023089F41630E9
:103E400079F48091080190910901009749F0019758
:103E5000909309018093080161E070E00E94D317FC
:103E600080E00E941120892BD9F770E8E72EF12C11
:103E7000EC22FD22C7FD06C0CE0180749270892B12
:103E800009F4FBCE41E060E981E00E942F24DD20AF
:103E900031F4612F645F40E050E08EE005C0602F98
:103EA0006C5E40E050E081E10E946830EF2861F0F4
:103EB000DD2021F4112359F1125016C0002311F412
:103EC00002E018C0025016C0C074D270CD2B51F061
:103ED000DD2021F41630E9F01E5F06C00230D9F073
:103EE0000E5F08C0DD2031F4612F645F43E350E0D2
:103EF0008EE005C0602F6C5E43E350E081E10E94DC
:103F0000683080E00E941120892BD9F7B6CE16E0E8
:103F1000EBCF10E0E9CF00E0EDCFDF92EF92FF9220
:103F20000F931F93CF93DF938BE194E00E94E520E2
:103F300089E594E00E94C13089E290E10E94C63098
:103F40000E943D1A43E350E06EE08FE00E9468302B
:103F500010E0DD24D39480E00E941120EC018870F1
:103F60009170892BA9F080E00E941120892BD9F74C
:103F7000143019F40E94D71D0BC0112319F41092AC
:103F80002C0104C0123021F4D0922C010E94891A15
:103F9000012F025F43E350E0602F8FE00E94683002
:103FA000E0E8EE2EF12CEC22FD22C7FD05C0CE018B
:103FB00080749270892B79F240E050E0602F8FE09E
:103FC0000E94683041E060E981E00E942F24EF28E0
:103FD00031F0112311F414E00BC0125009C0C07469
:103FE000D270CD2B29F0143011F410E001C01E5F07
:103FF000612F625F43E350E08FE00E94683080E011
:104000000E941120892BD9F7A6CF28E088E190E003
:104010000FB6F894A895809360000FBE20936000BF
:104020000895882329F48091AA0D9091AB0D04C0C6
:104030008091AC0D9091AD0D9093B4028093B3023A
:104040004091B3025091B4024F3F510519F1CA019A
:104050008070937080509340E9F4CA018870987022
:1040600088509840B9F48091AA0D9091AB0D892B9E
:1040700031F08091AC0D9091AD0D892BA1F728E026
:1040800088E190E00FB6F894A895809360000FBE89
:1040900020936000CA0108950F931F9383E09DE26F
:1040A0000E94E5200FE315E2C8010E94C630C80156
:1040B0000E94C1300E9400308FE090E00E94472EA5
:1040C00041E06FEF80E00E942F240FE81CE2A8017E
:1040D0006CE082E10E94FA2D83E090E00E94472E7E
:1040E00043EC5CE26CE082E10E94FA2D82E090E019
:1040F0000E94472EA8016CE082E10E94FA2D88E21E
:1041000090E00E94472E0E94003084E190E00E94DF
:10411000472E1F910F91089590E025E130E0829F96
:10412000F001839FF00D929FF00D1124EF54F24F98
:10413000618708956093DB04089590E025E130E005
:10414000829FF001839FF00D929FF00D1124EF5498
:10415000F24F12861182089590E025E130E0829FAF
:10416000F001839FF00D929FF00D1124EF54F24F58
:1041700081E0828B089590E025E130E0829FF0019C
:10418000839FF00D929FF00D1124EF54F24F608742
:10419000089590E025E130E0829FF001839FF00DCB
:1041A000929FF00D1124EF54F24F6483089590E034
:1041B00025E130E0829FF001839FF00D929FF00D8A
:1041C0001124EF54F24F658308959093080E809365
:1041D000070E1092B502E1EBFDE021E08FEF98E1D0
:1041E0002083178286831386808711829583759634
:1041F0003EE0E530F307A1F708951092B20D10925A
:10420000C70D1092DC0D1092F10D01969093100ED7
:1042100080930F0E9093B00D8093AF0D9093130E7B
:104220008093120E10920E0E10920D0E1092060E2A
:104230001092050E1092090E81E08093B502109243
:104240000C0E10920B0E08958091AF0D9091B00D51
:104250000E94FD2008958091BA0D87FD03C08AEF6A
:104260008093BA0D8091CF0D87FD03C08AEF8093B4
:10427000CF0D8091E40D87FD03C08AEF8093E40D9C
:104280008091F90D87FD03C08AEF8093F90D10929C
:10429000B502089581E08093B5020895DC01ED91A7
:1042A000FC911197AF014F5F5F4F11965C934E9356
:1042B000E4912E2F30E0E7FF13C02F773070369552
:1042C000322F222737952795FA014F5F5F4FE491F0
:1042D0008E2F8F77280F311DE7FDF1CF4D935C9323
:1042E000C901089508950F931F93CF93DF93182F5B
:1042F000062FEA01833049F481E091E09093DD04D8
:104300008093DC042093DB0410C0622F0E941F25E1
:10431000812F90E0FC01EE0FFF1FE80FF91FEE0F59
:10432000FF1FE853FB4FD283C183212F30E085E18B
:1043300090E0289FF001299FF00D389FF00D112487
:10434000EF54F24F81E082870783DF91CF911F9175
:104350000F9108950E941F250895EF92FF920F93E9
:104360001F93CF93DF93182F062FF42EE22EC82F22
:10437000D0E085E190E0C89FF001C99FF00DD89F83
:10438000F00D1124EF54F24F8285882321F08181B2
:10439000882309F077C0EE2091F485E190E0C89F72
:1043A000F001C99FF00DD89FF00D1124EF54F24F8A
:1043B000128A8185882309F065C0178263C0133093
:1043C00059F481E091E09093DD048093DC0481E076
:1043D0008093DB040F2D08C060E0812F0E941F2511
:1043E0006F2D812F0E9400250F3799F485E190E011
:1043F000C89FF001C99FF00DD89FF00D1124EF5414
:10440000F24F80910B0E86878CE09EE0948B838B1D
:1044100020C0802F90E0880F991FE091070EF09147
:10442000080EE80FF91F259134912F5F3F4FF901D6
:10443000449185E190E0C89FF001C99FF00DD89F9D
:10444000F00D1124EF54F24F46872F5F3F4F348B0E
:10445000238B85E190E0C89FF001C99FF00DD89FA4
:10446000F00D1124EF54F24F178611860387118245
:104470008FEF8087E782F282108A81E08287128A3A
:10448000118A1482DF91CF911F910F91FF90EF90CD
:104490000895CF92DF92FF920F931F93CF93DF93F4
:1044A000E9EBFDE08181282F332727FD30958081BE
:1044B000280F311D2F3F310519F014F02FEF30E098
:1044C000C90137FF02C080E090E0808375964EE01E
:1044D000ED30F40739F78091B502882309F0D9C08F
:1044E000F5C0E0910F0EF091100E9F012F5F3F4F2E
:1044F0003093100E20930F0E44914F3F69F5A901A0
:104500004F5F5F4F5093100E40930F0EF90184914F
:104510008F3219F41092B502CAC0863009F0AAC0D1
:10452000FA013196CF0101969093100E80930F0EF1
:10453000E491E33529F49093130E8093120E9AC000
:10454000E53409F097C08091120E9091130E90936C
:10455000100E80930F0E8EC047FF02C04093090ECD
:10456000542F5F70842F90E0807F9070803B910586
:1045700029F1803C910529F18039910509F038C075
:10458000C9010196F901449101969093100E809310
:104590000F0E0197FC012491852F90E08C9FF00174
:1045A0008D9FF00D9C9FF00D1124EF54F24F8081F0
:1045B000882309F45FC0220F638545C02E5F3F4FFB
:1045C00048C02F5F3F4F3093100E20930F0E2150A5
:1045D0003040F9012491852F90E08C9FF0018D9F50
:1045E000F00D9C9FF00D1124EF54F24F238742C031
:1045F0008091090E582F5F7090E0807F9070803B13
:10460000910529F1803C910549F18039910591F599
:104610002F5F3F4F3093100E20930F0E21503040EC
:10462000F9012491852F90E08C9FD0018D9FB00DD2
:104630009C9FB00D1124AF54B24F8C918823D1F0C0
:10464000220F1B966C91852F0E94AD2113C02F5F06
:104650003F4F3093100E20930F0E0CC0852F90E02B
:104660008C9FF0018D9FF00D9C9FF00D1124EF5455
:10467000F24F43878FE09EE00E944E2196958795EA
:1046800090930E0E80930D0E1092060E1092050E52
:1046900002C0C5E1D0E06091050E7091060E8091D8
:1046A0000D0E90910E0E6817790709F41ACF6F5FFF
:1046B0007F4F7093060E6093050E80910B0E9091C4
:1046C0000C0E019690930C0E80930B0E08EC14E0E8
:1046D000C2EBDDE0FF248FEFC82ED12C898988231F
:1046E00009F05EC08A899B89892B09F456C09E8592
:1046F0008D85981708F04CC050C08A852A893B895F
:104700008F37E9F4D9018D91BB8BAA8B8F3F01F1D3
:10471000F90161811196BB8BAA8BE82FF0E0EE0FB7
:10472000FF1FEE5EFE4F0190F081E02D8F2D099569
:10473000EA89FB8981918D87FB8BEA8B28C0A901CF
:104740004F5F5F4F5B8B4A8BF90184918F3F21F460
:1047500018821B8A1A8A21C04F5F5F4F5B8B4A8B7E
:1047600041505040FA016491E82FF0E0EE0FFF1F36
:10477000EE5EFE4F0190F081E02D8F2D0995EA89C4
:10478000FB893196FB8BEA8B3197E491ED871E868E
:104790009E858D85981709F4B0CF8E858F5F8E87A3
:1047A0008985882319F420E030E047C08F858F3F4A
:1047B00011F08F5F8F879E819923C9F12F8122236A
:1047C000B1F18D81882399F1899FC0011124805016
:1047D0009F4F892F992730E0AC01429FC001439F32
:1047E000900D529F900D112480509F4F292F3327F9
:1047F0008B818823F1F0EA81F0E0E050F24BE49104
:10480000E058E89FC001112480509F4F892F9927BD
:10481000F601E81BF90BE29FC001E39F900DF29FA8
:10482000900D112480509F4F292F332702C020E084
:1048300030E08A819C81890F8A83F8012083F39478
:104840000A5F1F4F6596F4E0FF1609F047CFDF912E
:10485000CF911F910F91FF90DF90CF9008951F93FC
:10486000CF93DF93582F90E0880F991F2091070E68
:104870003091080E280F391FF90185919491DC01C0
:104880001196FC018491813011F413E01DC08091D8
:10489000C70D8823B1F08091D20D851711F4442300
:1048A00081F48091DC0D882371F08091E70D8517EC
:1048B00011F4442341F49091D60D8091EB0D8917AA
:1048C00010F411E001C012E0212F30E0FD0144910D
:1048D00085E190E0289FE001299FD00D389FD00D01
:1048E0001124CF54D24F4E871196BC8BAB8B1F86B1
:1048F00080E58A836F838FEF888719861A8A188AE2
:1049000021E02A87198A5C8729831C82133049F4A5
:1049100081E091E09093DD048093DC042093DB043C
:1049200008C060E5812F0E9400256989812F0E94BF
:104930001F25DF91CF911F910895FF920F931F9331
:10494000082FF62E0E94002510E085E190E0089FD8
:10495000F001099FF00D189FF00D1124EF54F24F54
:10496000F2821F910F91FF900895962F482F50E0EB
:1049700025E130E0429FF001439FF00D529FF00D82
:104980001124EF54F24F6281691B62830E9400255B
:104990000895482F50E025E130E0429FF001439F09
:1049A000F00D529FF00D1124EF54F24F9281690FD8
:1049B00062830E94002508950000000000000000AE
:1049C00000000000000000000000000000000000E7
:1049D00000000000000000000000000000000000D7
:1049E00000000000000000000000000000000000C7
:1049F00000000000000000000000000000000000B7
:104A000099277727833008F00895E0E0F8E5660FEE
:104A1000771FE60FF71FA591B491E8ECF4E026E0CC
:104A2000289FE00DF11DA183B28311240895909178
:104A3000DB049170880F892B8093DB0408959927FC
:104A40007727E8ECF4E026E0289FE00DF11D6E3FAB
:104A500031F46091DB046E7F6093DB040BC06F3F29
:104A600031F46091DB046E6F6093DB0403C07EE47D
:104A7000760F75831124089599277727E8ECF4E0E1
:104A800026E0289FE00DF11D6083112408952F93E7
:104A90003F934F935F936F937F938F939F93AF93C6
:104AA000BF93789411240E94FE2E0E9449222F92D7
:104AB0003F924F925F926F927F928F929F92AF92AE
:104AC000BF92CF92DF92EF92FF920F931F93CF93FB
:104AD000DF930090C504002019F4A9EBB2E002C0F6
:104AE000AEEBB3E001E000260092C50402E00093C3
:104AF000C6042090C9043090CA044090CC04509061
:104B0000CD046090CB041091C8047090CF048090C5
:104B1000D0049090D104A090D204B090D3042091FE
:104B2000CE04C090D504D090D604E090D804F09084
:104B3000D9040091D7043091D4045091DA046091E3
:104B4000DC047091DD048091DE049FEF620C431C55
:104B5000F2014491410300240008C12DD02D970C8F
:104B6000A81CF5014491420300240008C10DD01D8A
:104B70000C0DED1CF7014491430300240008C10D06
:104B8000D01D8A956AF44091DB04842F8695062E09
:104B90000694062600FA7695679576F940FF66F941
:104BA00040E860FD4FE7450300240008C10DD01D1B
:104BB000D595C7950024C038D0050CF0CFE70A94EE
:104BC000C038D0050CF4C0E8CD939A9509F0BECF5B
:104BD0004091C6044A954093C60496E009F0B6CFCA
:104BE0006092CB044092CC049092D104A092D20463
:104BF0000093D704E092D8046093DC047093DD0442
:104C00008093DE04DF91CF911F910F91FF90EF9081
:104C1000DF90CF90BF90AF909F908F907F906F90DC
:104C20005F904F903F902F9099278091A00D77270C
:104C30006091A10D11240E947221BF91AF919F91AB
:104C40008F917F916F915F914F913F912F91089537
:104C5000A9EBB2E08AE092E000E00D930197E9F75A
:104C6000A9EBB2E0A093C304B093C404002700935F
:104C7000C5046EE46093CD046093D3046093D904BB
:104C800061E06093DC046093DD0461E06093DB0429
:104C900066276093C8046093CE046093D404609345
:104CA000DA046093C9046093CA046093CB046093F0
:104CB000CC046093CF046093D0046093D1046093DC
:104CC000D2046093D5046093D6046093D7046093B4
:104CD000D80411240895E091C304F091C404019113
:104CE00000580093B30004E0E33CF00709EB12E046
:104CF00008F0F801E093C304F093C40408950C9401
:104D000081260C9483260F931F932ABDE091C30440
:104D1000F091C404019100580093B30004E0E33C17
:104D2000F00710F40000000010F0E9EBF2E0E0936F
:104D3000C304F093C404C895C895C895C895C89590
:104D4000C8950000000000002AB51F910F9108953A
:104D50000000E091A10DE0FFD6CFE1E1EA95F1F787
:104D600000000000089500000000000000000000A6
:104D70000000000000000000000000000000000033
:104D80000000000000000000000000000000000023
:104D90000000000000000000000000000000000013
:104DA0000000000000000000000000000000000003
:104DB00000000000000000000000000000000000F3
:104DC00000000000000000000000000000000000E3
:104DD00000000000000000000000000000000000D3
:104DE00000000000000000000000000000000000C3
:104DF00000000000000000000000000000000000B3
:104E0000000306090C101316191C1F2225282B2E2F
:104E1000313336393C3F414447494C4E5153555844
:104E20005A5C5E60626466686A6B6D6F7071737401
:104E3000757678797A7A7B7C7D7D7E7E7E7F7F7FBA
:104E40007F7F7F7F7E7E7E7D7D7C7B7A7A797876A0
:104E500075747371706F6D6B6A68666462605E5CB6
:104E60005A585553514E4C494744413F3C393633CB
:104E7000312E2B2825221F1C191613100C0906038E
:104E800000FDFAF7F4F0EDEAE7E4E1DEDBD8D5D295
:104E9000CFCDCAC7C4C1BFBCB9B7B4B2AFADABA860
:104EA000A6A4A2A09E9C9A9896959391908F8D8C83
:104EB0008B8A8887868685848383828282818181AA
:104EC0008181818182828283838485868687888AA4
:104ED0008B8C8D8F9091939596989A9C9EA0A2A46E
:104EE000A6A8ABADAFB2B4B7B9BCBFC1C4C7CACD39
:104EF000CFD2D5D8DBDEE1E4E7EAEDF0F4F7FAFD56
:104F0000808182838485868788898A8B8C8D8E8F29
:104F1000909192939495969798999A9B9C9D9E9F19
:104F2000A0A1A2A3A4A5A6A7A8A9AAABACADAEAF09
:104F3000B0B1B2B3B4B5B6B7B8B9BABBBCBDBEBFF9
:104F4000C0C1C2C3C4C5C6C7C8C9CACBCCCDCECFE9
:104F5000D0D1D2D3D4D5D6D7D8D9DADBDCDDDEDFD9
:104F6000E0E1E2E3E4E5E6E7E8E9EAEBECEDEEEFC9
:104F7000F0F1F2F3F4F5F6F7F8F9FAFBFCFDFEFFB9
:104F8000000102030405060708090A0B0C0D0E0FA9
:104F9000101112131415161718191A1B1C1D1E1F99
:104FA000202122232425262728292A2B2C2D2E2F89
:104FB000303132333435363738393A3B3C3D3E3F79
:104FC000404142434445464748494A4B4C4D4E4F69
:104FD000505152535455565758595A5B5C5D5E5F59
:104FE000606162636465666768696A6B6C6D6E6F49
:104FF000707172737475767778797A7B7C7D7E7F39
:1050000000020406080A0C0E10121416181A1C1EB0
:1050100020222426282A2C2E30323436383A3C3EA0
:1050200040424446484A4C4E50525456585A5C5E90
:1050300060626466686A6C6E70727476787A7C7E80
:105040007F7D7B79777573716F6D6B696765636160
:105050005F5D5B59575553514F4D4B494745434150
:105060003F3D3B39373533312F2D2B292725232140
:105070001F1D1B19171513110F0D0B090705030130
:10508000FFFDFBF9F7F5F3F1EFEDEBE9E7E5E3E120
:10509000DFDDDBD9D7D5D3D1CFCDCBC9C7C5C3C110
:1050A000BFBDBBB9B7B5B3B1AFADABA9A7A5A3A100
:1050B0009F9D9B99979593918F8D8B8987858381F0
:1050C00080828486888A8C8E90929496989A9C9EF0
:1050D000A0A2A4A6A8AAACAEB0B2B4B6B8BABCBEE0
:1050E000C0C2C4C6C8CACCCED0D2D4D6D8DADCDED0
:1050F000E0E2E4E6E8EAECEEF0F2F4F6F8FAFCFEC0
:105100007F7F7F7F7F7F7F7F7F7F7F7F7F7F7F7FAF
:105110007F7F7F7F7F7F7F7F7F7F7F7F7F7F7F7F9F
:105120007F7F7F7F7F7F7F7F7F7F7F7F7F7F7F7F8F
:105130007F7F7F7F7F7F7F7F7F7F7F7F7F7F7F7F7F
:105400000309131E28313A40464C5054585B5E61E4
:10541000636567696B6C6E6F7071727374757677A4
:10542000777879797A7A7B7B7C7C7C7D7D7D7E7ECA
:105430007E7E7F7F7F7F7F7F7F7F7F7F7F7F7F7F7E
:105440007F7F7F7F7F7F7F7F7F7F7F7F7F7E7E7E6F
:105450007E7D7D7D7C7C7C7B7B7A7A7979787777A1
:10546000767574737271706F6E6C6B69676563616A
:105470005E5B5854504C46403A31281E13090300D5
:10548000C6CCD5DBDFE3E5E7E9EAEBECEDEEEFEFE9
:10549000F0F0F0F1F1F1F1F2F2F2F2F2F2F2F2F3F5
:1054A000F3F3F3F3F3F3F3F3F3F3F3F3F3F3F3F3CC
:1054B000F3F3F3F3F3F3F3F3F3F3F3F3F3F3F3F3BC
:1054C000F3F3F3F3F3F3F3F3F3F3F3F3F3F3F3F3AC
:1054D000F3F3F3F3F3F3F3F3F3F3F3F3F3F3F3F39C
:1054E000F2F2F2F2F2F2F2F2F1F1F1F1F0F0F0EFA9
:1054F000EFEEEDECEBEAE9E7E5E3DFDBD5CCC60068
:1055000000283D42302D2C2B2C2D2E2F30323335C0
:1055100037393B3D3F414345484A4C4E5053555720
:10552000595B5D5F61636567696B6C6E7071737405
:10553000757778797A7B7C7D7D7E7E7F7F7F7F7FAC
:105540007F7F7F7F7F7F7E7E7D7D7C7B7A79787792
:1055500075747371706E6C6B69676563615F5D5BB9
:1055600059575553504E4C4A484543413F3D3B39AE
:1055700037353332302F2E2D2C2B2C2D30423D2819
:1055800000E9E5FED4D7D7D7D6D4D2D0CECCCAC87E
:10559000C6C3C1BFBDBAB8B6B4B1AFADABA9A7A5BC
:1055A000A3A19F9E9C9A999795949391908F8D8C8F
:1055B0008B8A89888887868585848484838383838E
:1055C0008383838383848484858586878888898A86
:1055D0008B8C8D8F909193949597999A9C9E9FA177
:1055E000A3A5A7A9ABADAFB1B4B6B8BABDBFC1C38F
:1055F000C6C8CACCCED0D2D4D6D7D7D7D4FEE5E948
:10560000F9F8F9F5EBE1DDDEE0E2E4E5E6E5E4E218
:10561000DED9D2CAC1B7ACA299918A868381808033
:105620008182838586888A8C8D8F909293959697B8
:1056300098999A9B9B9C9D9D9D9E9E9E9F9F9F9FA0
:105640009F9F9F9E9E9E9D9D9D9C9B9B9A99989798
:1056500096959392908F8D8C8A888685838281809F
:10566000808183868A9199A2ACB7C1CAD2D9DEE281
:10567000E4E5E6E5E4E2E0DEDDE1EBF5F9F8F9008A
:105680000708070B151F2322201E1C1B1A1B1C1E9C
:1056900022272E363F49545E676F767A7E7F7F7F62
:1056A0007F7E7D7B7A7876747371706E6D6B6A69BC
:1056B00068676665656464636362626261616161B3
:1056C000616161626262636363646565666768699C
:1056D0006A6B6D6E7071737476787A7B7D7E7F7F76
:1056E0007F7F7E7A766F675E54493F362E27221E73
:1056F0001C1B1A1B1C1E2022231F150B070807004A
:105700001F313D444E5354565A5F64696E74767926
:105710007C7F7F7F7F7F7F7F7F7F7F7F7F7F7F7F9C
:105720007F7F7F7F7F7F7F7F7F7F7F7F7F7F7F7F89
:105730007F7F7F7F7F7F7F7F7F7F7F7F7F7F7F7F79
:105740007F7F7F7F7F7F7F7F7F7F7F7F7F7F7F7F69
:105750007F7F7F7F7F7F7F7F7F7F7F7F7F7F7F7F59
:105760007F7F7F7F7F7F7F7F7F7F7F7F7F7F7F7F49
:105770007F7F7F7F7F7F7F7F7F7F7F7C7871684C9B
:105780002C1C120C0A0B0A05FDF3E9DFD4CAC0B7C2
:10579000AEA69E97918B8685828080808080808057
:1057A00080808080808080808080808080808080F9
:1057B00080808080808080808080808080808080E9
:1057C00080808080808080808080808080808080D9
:1057D00080808080808080808080808080808080C9
:1057E00080808080808080808080808080808080B9
:1057F000808080808087919DACC4CBD4DDF2FAFAA2
:1058000022002400260028002B002D003000330049
:10581000360039003D004000440048004C00510073
:1058200056005B00600066006C0073007900810028
:10583000880090009900A200AC00B600C100CC0026
:10584000D800E500F30001011001210132014401FB
:1058500057016C0181019801B001CA01E501020202
:105860002102410264028802AE02D7020303300320
:1058700061039403CB03050442048304C7041005A9
:105880005D05AF0505066106C206290796070908EA
:10589000830805098E09200ABA0A5D0B0A0CC10C9F
:1058A000840D510E2B0F121007110A121D134014F4
:1058B0007415BA1614188319071BA31C571E24202D
:1058C0000E22142439267F28E82A752D2930063324
:1058D0000F364539AD3C49401B442848734CFE50B7
:1058E000CF55EA5A51600C661D6C8B725A799280C2
:1058F00037885090E598FDA19FABD3B5A3C00000B9
:105900001F93CF93DF93FA01549131961491C52FD1
:10591000D0E09F012F5F3F4F70E095E0660F771F4B
:105920009A95E1F7680F711D40E00FC084918C9348
:1059300011961C9211979F5F319612969517B0F3AE
:105940004F5F2C0F3D1F605E7F4F411740F4DB011E
:10595000AA0FBB1FA052BB4FF90190E0EFCFDF9120
:10596000CF911F9108958F929F92AF92BF92CF9245
:10597000DF92EF92FF920F931F93CF93DF93882EC6
:10598000962E5A016901F02E00E010E080EEF80E2C
:105990000CC04F2D6E2D882D8C0F0E9450302196FB
:1059A000CA15DB05B4F30F5F1F4F0C151D052CF452
:1059B000C0E0D0E0E02EE90CF3CFDF91CF911F9152
:1059C0000F91FF90EF90DF90CF90BF90AF909F909E
:1059D0008F90089540520E9450300895FF920F9387
:1059E0001F93CF93DF938C01F62EEA01FE014491C1
:1059F0002196442349F0802F0F5F1F4F4F7740526D
:105A00006F2D0E945030F2CFDF91CF911F910F91F7
:105A1000FF900895FF920F931F93182F062FF42ED7
:105A200042954F704A3010F4405F01C0495E602FCC
:105A3000812F0E9450304F2D4F70812F8F5F4A3041
:105A400010F4405F01C0495E602F0E9450301F91EA
:105A50000F91FF900895FF920F931F93F82E162F2A
:105A6000042F452F0E940A2D402F612F8F2D8E5F0E
:105A70000E940A2D1F910F91FF900895EF92FF92BF
:105A80000F931F93F62E042F182F28E0E22EE80E16
:105A900007FF02C041E101C040E16F2D812F0E944C
:105AA00050301F5F1E1511F0000FF2CF1F910F91A4
:105AB000FF90EF900895FF920F931F93CF93DF9382
:105AC000F62E042FEC0110E0002311F4112339F419
:105AD000802F6AE00E945231905F492F01C040E060
:105AE0006F2D8C2F0E9450301F5F2197133031F0A3
:105AF000802F6AE00E945231082FE6CFDF91CF91CC
:105B00001F910F91FF900895CF92DF92EF92FF9235
:105B10000F931F93CF93DF93C62E79018A01EC0177
:105B2000DD24E114F1040105110511F4DD2059F41F
:105B3000C801B7012AE030E040E050E00E94713136
:105B4000462F405F01C040E06C2D8C2F0E945030EA
:105B5000D394219786E0D81669F0C801B7012AE0EE
:105B600030E040E050E00E947131C901DA017C016F
:105B70008D01D7CFDF91CF911F910F91FF90EF90C3
:105B8000DF90CF9008957F928F929F92AF92BF92B5
:105B9000CF92DF92EF92FF920F931F93CF93DF93F9
:105BA000782E862E5A016901780100E010E00CC0C1
:105BB000A701692D872D8C0F0E9468302196CA1588
:105BC000DB05B4F30F5F1F4F0C151D052CF4C0E06F
:105BD000D0E0902E980CF3CFDF91CF911F910F91D1
:105BE000FF90EF90DF90CF90BF90AF909F908F90FD
:105BF0007F9008957F928F929F92AF92BF92CF92A3
:105C0000DF92EF92FF920F931F93CF93DF93782E43
:105C1000862EEA01FA01C590D490FA013296A59039
:105C2000B49000E016C0FC01EE0DFF1D3296EE0FA1
:105C3000FF1FEC0FFD1F45915491692D812F870D9A
:105C40000E9468301F5F812F90E08C159D055CF3EA
:105C50000F5F802F90E08A159B055CF48C9D70018E
:105C60008D9DF00C9C9DF00C112410E0902E980C52
:105C7000EACFDF91CF911F910F91FF90EF90DF90CE
:105C8000CF90BF90AF909F908F907F9008950F938B
:105C90001F93CF93DF938C01C0E0D0E007C00E9438
:105CA000D0308823E1F30E94D3302196C017D1076A
:105CB000B4F3DF91CF911F910F910895BE2FC82F9C
:105CC000D62FEC2ECC03CC03CC03CC03CC03CC03DB
:105CD000CC03CC03CC03CC03CC03CC03CC03CC034C
:105CE000CC03CC03CC03CC03CC03CC03CC03CC033C
:105CF000CC03CC03CC03CC03CC03CC03CC03CC032C
:105D0000CC03CC03CC03CC03CC03CC03CC03CC031B
:105D1000CC03CC03CC03CC03CC03CC03CC03CC030B
:105D2000CC03CC03CC03CC0386E891E00197F1F7D8
:105D30000000C0EED4E070EE662711D134E23A954F
:105D4000F1F70E94CC2E3BE13A95F1F700007A95ED
:105D500089F0C8956395683029F0C895C895C895AD
:105D60000000EBCF662730E5C30FD61FC8950000B3
:105D70000000E3CF35E03A95F1F700C0F0D011E034
:105D80000091A30D01270093A30D00FF1093A20D16
:105D9000E2E0E09336000895DE0106E0609FED91B9
:105DA000FD91E00DF11D18E2059108B94D910591A5
:105DB00008B95D91059108B9400D511D059108B9CB
:105DC00000C0059108B90591FA011A9508B961F763
:105DD000C895002708B9089528980E947F26E7E112
:105DE000EA95F1F7289A05D1E0E0F6E0E8D0E0FF87
:105DF00043D0E0FF02C00E9447250895129A0C94F8
:105E0000012F0C94032F12984427552766277727D4
:105E10008CE00C940B2F0C940D2F0C940F2F0C94E2
:105E2000112F0C94132F0C94152F440F551F00990C
:105E30004160660F771F01996160139A0C94202FBF
:105E40000C94222F13980C94252F0C94272F0C942C
:105E5000292F0C942B2F8A9541F7409550956095EA
:105E600070955F707F704093AA0D5093AB0D609357
:105E7000AC0D7093AD0D0895EF93E091A10DE83E48
:105E8000E0F5E830D0F12F923F924F925F926F92FF
:105E90007F928F929F92AF92BF92CF92DF92EF92BA
:105EA000FF920F931F932F933F934F935F936F93A3
:105EB0007F938F939F93AF93BF93CF93DF930E9472
:105EC000942EDF91CF91BF91AF919F918F917F9150
:105ED0006F915F914F913F912F911F910F91FF9083
:105EE000EF90DF90CF90BF90AF909F908F907F907A
:105EF0006F905F904F903F902F90EF910895FF9398
:105F0000EF93EFB7EF93E0918400EE50E13000F0B3
:105F1000E23000F0E33000F0E43000F0E53000F073
:105F2000E63000F0E73000F0E83000F0E93000F053
:105F300005D0EF91EFBFEF91FF9118950F921F924F
:105F4000ECEBFCE50090A00D000C1124E00DF11D20
:105F500005901490F00109951F900F9008952898CE
:105F60000E947F26E5E1EA95F1F7E091A10DEA951F
:105F7000E093A10D289A00000000089528980E943F
:105F8000A826289A0000E1E0F6E019D02BD0089569
:105F900028980E94A826E0EB0000EA95E9F70000A7
:105FA0000000289AF6E0E2E00AD0089528980E94BE
:105FB000A826289A0000E3E0FCEF01D008950090A5
:105FC000A10D0A9410905F0011FC0F2E0092A10DFC
:105FD0000090A00D11FC0E2E0092A00DE0E011FC2F
:105FE000E1E00895E3E0E0938900EDE8E0938800C4
:105FF0000895E7E0E0938900EBE1E09388000895DD
:10600000E0E6F4E0A0EEB4E06091A80D7091A90D77
:106010006D937D933197E1F7112408950F931F93AA
:1060200080E694E0A0EEB4E0E091A60DF091A70D1B
:1060300040E30091A40D1091A50D65917591649FA9
:106040009001749F300D200F311F2D933D930197C8
:10605000A1F711241F910F910895992777273327CE
:1060600020E5629F880F080E131EE091A60DF091A7
:10607000A70DE00DF11D45915591A0EEB4E0A00DE6
:10608000B11D20E3429FB001529F700D4091A40DBD
:106090005091A50D640F751F6D937C931124089585
:1060A0009927552728E2220F629F880F080E191E94
:1060B000A0EEB4E0A00DB11D6091A80D7091A90DE6
:1060C00020E3429F600D711D6D937C931124089510
:1060D0009927772728E2220F629F880F080E191E42
:1060E000A0EEB4E0A00DB11D6091A40D7091A50DBE
:1060F00020E3429F600D711D529F700D6D937C9344
:1061000011240895F894442740938100409345005A
:106110004FEF47B944B940E84AB941E04C7F4C6081
:1061200041B91298139800E00093A00D06E0009387
:10613000A10D409385004093840043E04093890083
:106140004DE84093880049E04093810042E040934D
:106150006F0042E44093440040E04093470041E038
:1061600000004093450043E84093B00040E0409376
:10617000B30041E04093B10041E045B97894112467
:1061800008958093A80D9093A90D08958093A40D70
:106190009093A50D08958093A60D9093A70D089553
:1061A0008091A20D089511241092A20D08958823C4
:1061B00029F48091AA0D9091AB0D08958091AC0DBA
:1061C0009091AD0D089580E891E0809361009093E7
:1061D0006100089580E890E08093610090936100F1
:1061E0000895A0E0B0E0E7EFF0E30C94E931EC01B2
:1061F000A880B980CA80DB80A114B104C104D10495
:1062000041F484E2A82E89EDB82E8BE5C82E87E0F4
:10621000D82EC601B5012DE133EF41E050E00E94D8
:10622000C63127EA31E440E050E00E94A7317B010B
:106230008C01C601B5012DE133EF41E050E00E9431
:10624000C631CA01B9012CEE34EF4FEF5FEF0E9467
:10625000A7316E0D7F1D801F911F97FF04C06150F5
:10626000704080409048688379838A839B839B0138
:106270003F77C901CDB7DEB7EAE00C9405320E9442
:10628000F130089588E291E00E94F1300895A0E095
:10629000B0E08093280190932901A0932A01B09344
:1062A0002B010895991B79E004C0991F961708F0F7
:1062B000961B881F7A95C9F78095089597FB092E3C
:1062C00007260AD077FD04D02ED006D000201AF47D
:1062D000709561957F4F0895F6F7909581959F4F42
:1062E0000895A1E21A2EAA1BBB1BFD010DC0AA1F17
:1062F000BB1FEE1FFF1FA217B307E407F50720F02F
:10630000A21BB30BE40BF50B661F771F881F991FA9
:106310001A9469F760957095809590959B01AC01F2
:10632000BD01CF010895AA1BBB1B51E107C0AA1FE5
:10633000BB1FA617B70710F0A61BB70B881F991F26
:106340005A95A9F780959095BC01CD010895629F5B
:10635000D001739FF001829FE00DF11D649FE00D5D
:10636000F11D929FF00D839FF00D749FF00D659FBE
:10637000F00D9927729FB00DE11DF91F639FB00DBD
:10638000E11DF91FBD01CF011124089597FB092ECE
:1063900005260ED057FD04D0A4DF0AD0001C38F427
:1063A00050954095309521953F4F4F4F5F4F089541
:1063B000F6F790958095709561957F4F8F4F9F4F21
:1063C00008952F923F924F925F926F927F928F9299
:1063D0009F92AF92BF92CF92DF92EF92FF920F9374
:1063E0001F93CF93DF93CDB7DEB7CA1BDB0B0FB67E
:1063F000F894DEBF0FBECDBF09942A88398848883B
:106400005F846E847D848C849B84AA84B984C884D0
:10641000DF80EE80FD800C811B81AA81B981CE0FC7
:10642000D11D0FB6F894DEBF0FBECDBFED010895AC
:04643000F894FFCF0E
:10643400020003000A0A0300020001000A000F0020
:1064440001008C209A20AA21C924B5249D20AC20C7
:0C645400BB209D24C920D72001000000BF
:00000001FF
